:020000040000FA
:06000000FEEF02F0120009
:02002A000000D4
:04002C00806AF80EE0
:10003000926E070EC16E809080948092936A120037
:1000400093688082809400008084000081BEFAD78B
:10005000809400008092936A1200D9CFE6FFE1CF2E
:10006000D9FF80928090FE0EDB50816EE9DF8080A8
:10007000808400008094010EE66E0AEC03F0E552E5
:10008000E552E7CFD9FF1200D9CFE6FFE1CFD9FF84
:1000900080928090FE0EDB50816ED2DF8084000063
:1000A0008094010EE66E0AEC03F0E552E552E7CFCC
:1000B000D9FF12003C0EE66EE7DFE5520B0EE66E4E
:1000C000F0EC02F0E5523C0EE66EDEDFE5520B0E80
:1000D000E66EF0EC02F0E5523C0EE66ED5DFE5523E
:1000E0000B0EE66EF0EC02F0E552080EE66ECCDF89
:1000F000E552010EE66EC8DFE552060EE66EC4DF7D
:10010000E5521200F00E936EF19E816A81380F0B5A
:1001100000018D6F8C6B8DA104D08D918D438C2B44
:10012000FAD7040E8C5D1CE28CC08EF00F0E936E1D
:10013000F19E816A81148D6F8C6B8DA104D08D919D
:100140008D438C2BFAD7040E8C5D08E28CC08DF0A9
:100150008E51040DF3508D258A6F01D08A6901D02C
:100160008A691200260EE66EE66A3C0EE66E3CECEC
:1001700002F0E552E552E5521200D9CFE6FFE1CF99
:10018000D9FFACA2FED7FE0EDBCFE6FFD9EC02F022
:10019000E552E552E7CFD9FF1200C750040B11E139
:1001A000C550100B0EE1C550080B0BE1C550040BF8
:1001B00008E1C550020B05E1C550010B02E1000E3C
:1001C00001D0010E00D0120094680E0EC86EC00E51
:1001D000E66E080EE66E8FEC02F0E552E552120074
:1001E000C5801200C5841200D9CFE6FFE1CFD9FF48
:1001F000D4DF000901E0FCD7FE0EDBCFE6FFAAEC5E
:1002000002F0E552E552E7CFD9FF1200C6DF000940
:1002100001E0FCD7C750010B02E0000E01D0010E37
:10022000C586C7A0FED7C95000D01200D9CFE6FFBF
:10023000E1CFD9FFF70E9E149E6EFE0EDB5004E058
:10024000200EC510C56E03D0DF0EC514C56E100E8E
:10025000C510C56E9EA6FED7E552E7CFD9FF1200A6
:10026000E5DE28DF3C0EE66E0FDFE5520F0EE66E90
:100270000BDFE552826A00018F6B74DFA5DF00019E
:10028000906B8A6B0F0E00018A5D47E09EAA08D032
:1002900070EC02F000018B6F8BC0E6FFDEDEE552F2
:1002A00031DF100E00018A5D2FE28F512CE1010E2B
:1002B0008F6F0A0E8A5D0CE2300E8A25E66ECDDE67
:1002C000E552300E00018A25E66E57DFE5520BD06D
:1002D000370E8A25E66EC1DEE552370E00018A250B
:1002E000E66E4BDFE5527CDFA00EE66E7DDFE55269
:1002F00090C0E6FF79DFE5528AC0E6FF75DFE55280
:1003000071DF0001902B03D08F5101E08F6B020E43
:10031000E66EC2EC02F0E552B5D7C00EE66EB4DE72
:10032000E5520001906B50DF5BDFA00EE66E5CDFF4
:10033000E55290C0E6FF58DFE55254DF51DFA10ED1
:10034000E66E52DFE55200018A6B906B0F0E8A5DFC
:100350003DE0040E905D3AE215EC03F000018A6F77
:100360008A390F0B916F0A0E915D06E2300E9125CE
:10037000E66E73DEE55205D0370E9125E66E6DDE32
:10038000E5520F0E00018A15916F0A0E915D06E28B
:10039000300E9125E66E61DEE55205D0370E9125CF
:1003A000E66E5BDEE5522D0EE66E57DEE5520F0E71
:1003B00000018A5D05E1010EE66E38DFE55203D0EB
:1003C000E66A34DFE5520001902BC0D70BDF020E46
:0A03D000E66E5ADEE55253D7120024
:0603DA002A0EF66E000E73
:1003E000F76E000EF86E00010900F550856F0900E8
:1003F000F550866F03E1856701D03DD00900F550C7
:10040000806F0900F550816F0900F550826F090077
:100410000900F550E96E0900F550EA6E090009007F
:100420000900F550836F0900F550846F0900090039
:10043000F6CF87F0F7CF88F0F8CF89F080C0F6FFCD
:1004400081C0F7FF82C0F8FF0001835302E18453AB
:1004500007E00900F550EE6E8307F8E28407F9D74C
:1004600087C0F6FF88C0F7FF89C0F8FF0001850745
:08047000000E865BBFD71200ED
:08047800D9CFE6FFDACFE6FF61
:10048000E1CFD9FFE2CFDAFFAC6AAB6AFD0EDBB099
:10049000AC88DBA202D0AC8CAB8CDBB4AC8EDBA620
:1004A00002D0AB8801D0AB8ADBA802D0AC8401D0EB
:1004B000AC949E98DBAC02D09D8A01D09D9A9E9A06
:1004C000DBAE02D09D8801D09D98FB0EDB50AF6E55
:1004D000AC8AAB8EE552E5CFDAFFE7CFD9FF120049
:1004E000D9CFE6FFDACFE6FFE1CFD9FFE2CFDAFFDF
:1004F000E652F00E00019217ABAC03D09291ABB074
:100500009281ABB49285ABB29287AE50DF6EDF5072
:0E051000E552E552E5CFDAFFE7CFD9FF120042
:02051E00D9CF33
:10052000E6FFDACFE6FFE1CFD9FFE2CFDAFF3F0EF9
:10053000C716C66AC56AFD0EDB50C612FC0EDB503C
:10054000C71294869488C68AE552E5CFDAFFE7CFD2
:04055000D9FF1200BD
:0C055400D9CFE6FFDACFE6FFE1CFD9FFF8
:10056000E2CFDAFFFD0EDB50C96EC6AE02D0FF0E41
:1005700003D0C7B0FED7000EE552E5CFDAFFE7CFD4
:04058000D9FF12008D
:0C058400FF0EE350036EEF0E01D0F30EEB
:10059000E76EE72EC9EF02F00C0E026EE76AE72E57
:1005A000CFEF02F0022ECEEF02F0032EC7EF02F0E3
:0205B000120037
:0E05B200D9CFE6FFDACFE6FFE1CFD9FFE2CFE7
:1005C000DAFFACAC04D0AC90000192B3AC80FD0E6D
:1005D000DB50AD6EE552E5CFDAFFE7CFD9FF120071
:1005E000FF0EE350036E1B0E00D001D0200EE76E0D
:0C05F000E72EFED7032EFAD700D0120031
:0405FC0015EE00F008
:1006000025EE00F0F86A019CEDEC01F030EC01F011
:04061000FDD7120000
:0C061400FF0EE350E84E1200000000D082
:0A06200000D000D0E82EFAD7120037
:06062A00C586C7A0FED743
:04063000C95012009B
:020000040030CA
:0E00000000220F0E000181000FC00FE00F4024
:00000001FF
